:020000040801F1
:100000000000022049290108D1110108D31101087B
:10001000D5110108D7110108D9110108000000000D
:10002000000000000000000000000000DB110108DB
:10003000DD11010800000000DF110108E1110108D5
:100040009929010899290108992901089929010884
:100050009929010899290108992901089929010874
:100060009929010899290108992901089929010864
:100070009929010899290108992901089929010854
:100080009929010899290108992901089929010844
:100090009929010899290108992901089929010834
:1000A0009929010899290108992901089929010824
:1000B0009929010899290108992901089929010814
:1000C0009929010899290108992901089929010804
:1000D00099290108E9110108F91101089929010874
:1000E00099290108992901089929010899290108E4
:1000F00099290108992901089929010899290108D4
:1001000099290108992901089929010899290108C3
:10011000091201089929010899290108992901085A
:1001200099290108992901089929010899290108A3
:100130009929010899290108992901089929010893
:100140009929010899290108992901089929010883
:100150009929010899290108992901089929010873
:100160009929010899290108992901089929010863
:10017000992901089929010899290108000000001E
:080180009929010899290108E1
:1001880010B5054C237833B9044B13B10448AFF3C9
:1001980000800123237010BD18000020000000001B
:1001A800F429010808B5034B1BB103490348AFF311
:1001B800008008BD000000001C000020F429010890
:1001C80081F0004102E000BF83F0004330B54FEA00
:1001D80041044FEA430594EA050F08BF90EA020F6D
:1001E8001FBF54EA000C55EA020C7FEA645C7FEA00
:1001F800655C00F0E2804FEA5454D4EB5555B8BF23
:100208006D420CDD2C4480EA020281EA030382EA93
:10021800000083EA010180EA020281EA0303362D25
:1002280088BF30BD11F0004F4FEA01314FF4801CF8
:100238004CEA113102D0404261EB410113F0004F0A
:100248004FEA03334CEA133302D0524263EB4303C1
:1002580094EA050F00F0A780A4F10104D5F1200E5F
:100268000DDB02FA0EFC22FA05F2801841F10001BA
:1002780003FA0EF2801843FA05F359410EE0A5F18E
:1002880020050EF1200E012A03FA0EFC28BF4CF0BF
:10029800020C43FA05F3C01851EBE37101F0004575
:1002A80007D54FF0000EDCF1000C7EEB00006EEB82
:1002B8000101B1F5801F1BD3B1F5001F0CD349080C
:1002C8005FEA30004FEA3C0C04F101044FEA445263
:1002D80012F5800F80F09A80BCF1004F08BF5FEAEA
:1002E800500C50F1000041EB045141EA050130BDCA
:1002F8005FEA4C0C404141EB0101013C28BFB1F5DC
:10030800801FE9D291F0000F04BF01460020B1FA26
:1003180081F308BF2033A3F10B03B3F120020CDAF9
:100328000C3208DD02F1140CC2F10C0201FA0CF0D7
:1003380021FA02F10CE002F11402D8BFC2F1200C3C
:1003480001FA02F120FA0CFCDCBF41EA0C019040F2
:10035800E41AA2BF01EB0451294330BD6FEA04043B
:100368001F3C1CDA0C340EDC04F11404C4F1200226
:1003780020FA04F001FA02F340EA030021FA04F338
:1003880045EA030130BDC4F10C04C4F1200220FA8F
:1003980002F001FA04F340EA0300294630BD21FACD
:1003A80004F0294630BD94F0000F83F4801306BF93
:1003B80081F480110134013D4EE77FEA645C18BF87
:1003C8007FEA655C29D094EA050F08BF90EA020F1E
:1003D80005D054EA000C04BF1946104630BD91EA16
:1003E800030F1EBF0021002030BD5FEA545C05D119
:1003F8004000494128BF41F0004130BD14F5800458
:100408003CBF01F5801130BD01F0004545F0FE41CB
:1004180041F470014FF0000030BD7FEA645C1ABF00
:10042800194610467FEA655C1CBF0B46024650EA37
:10043800013406BF52EA033591EA030F41F4002163
:1004480030BD00BF90F0000F04BF0021704730B5E9
:100458004FF4806404F132044FF000054FF00001BE
:1004680050E700BF90F0000F04BF0021704730B57F
:100478004FF4806404F1320410F0004548BF404254
:100488004FF000013EE700BF42004FEAE2014FEAA9
:1004980031014FEA02701FBF12F07F4393F07F4F84
:1004A80081F06051704732F07F4208BF704793F087
:1004B8007F4F04BF41F40021704730B54FF460749A
:1004C80001F0004521F000411CE700BF50EA01029D
:1004D80008BF704730B54FF000050AE050EA010246
:1004E80008BF704730B511F0004502D5404261EBB6
:1004F80041014FF4806404F132045FEA915C3FF4F7
:10050800D8AE4FF003025FEADC0C18BF03325FEA93
:10051800DC0C18BF033202EBDC02C2F1200300FA44
:1005280003FC20FA02F001FA03FE40EA0E0021FA69
:1005380002F11444BDE600BF70B54FF0FF0C4CF457
:10054800E06C1CEA11541DBF1CEA135594EA0C0F09
:1005580095EA0C0F00F0DEF82C4481EA030621EA44
:100568004C5123EA4C5350EA013518BF52EA03357F
:1005780041F4801143F4801338D0A0FB02CE4FF031
:100588000005E1FB02E506F00042E0FB03E54FF061
:100598000006E1FB03569CF0000F18BF4EF0010E59
:1005A800A4F1FF04B6F5007F64F5407404D25FEA55
:1005B8004E0E6D4146EB060642EAC62141EA555108
:1005C8004FEAC52040EA5E504FEACE2EB4F1FD0C4A
:1005D80088BFBCF5E06F1ED8BEF1004F08BF5FEAC8
:1005E800500E50F1000041EB045170BD06F000467A
:1005F80046EA010140EA020081EA0301B4EB5C0427
:10060800C2BFD4EB0C0541EA045170BD41F480111E
:100618004FF0000E013C00F3AB8014F1360FDEBF43
:10062800002001F0004170BDC4F10004203C35DA1F
:100638000C341BDC04F11404C4F1200500FA05F3A2
:1006480020FA04F001FA05F240EA020001F0004243
:1006580021F0004110EBD37021FA04F642EB0601B9
:100668005EEA430E08BF20EAD37070BDC4F10C04E3
:10067800C4F1200500FA04F320FA05F001FA04F2A7
:1006880040EA020001F0004110EBD37041F1000193
:100698005EEA430E08BF20EAD37070BDC4F120059E
:1006A80000FA05F24EEA020E20FA04F301FA05F206
:1006B80043EA020321FA04F001F0004121FA04F2AE
:1006C80020EA020000EBD3705EEA430E08BF20EA7E
:1006D800D37070BD94F0000F0FD101F000464000B8
:1006E80041EB010111F4801F08BF013CF7D041EA3A
:1006F800060195F0000F18BF704703F0004652003E
:1007080043EB030313F4801F08BF013DF7D043EA0E
:100718000603704794EA0C0F0CEA135518BF95EAC4
:100728000C0F0CD050EA410618BF52EA4306D1D14B
:1007380081EA030101F000414FF0000070BD50EA6A
:10074800410606BF1046194652EA430619D094EAF4
:100758000C0F02D150EA013613D195EA0C0F05D1DE
:1007680052EA03361CBF104619460AD181EA030132
:1007780001F0004141F0FE4141F470014FF00000EA
:1007880070BD41F0FE4141F4780170BD70B54FF085
:10079800FF0C4CF4E06C1CEA11541DBF1CEA135505
:1007A80094EA0C0F95EA0C0F00F0A7F8A4EB0504E7
:1007B80081EA030E52EA03354FEA013100F08880DE
:1007C8004FEA03334FF0805545EA131343EA1263A7
:1007D8004FEA022245EA111545EA10654FEA00265C
:1007E8000EF000419D4208BF964244F1FD0404F515
:1007F800407402D25B084FEA3202B61A65EB030571
:100808005B084FEA32024FF480104FF4002CB6EB2D
:10081800020E75EB030E22BFB61A754640EA0C00AD
:100828005B084FEA3202B6EB020E75EB030E22BFED
:10083800B61A754640EA5C005B084FEA3202B6EB2E
:10084800020E75EB030E22BFB61A754640EA9C00ED
:100858005B084FEA3202B6EB020E75EB030E22BFBD
:10086800B61A754640EADC0055EA060E18D04FEA7B
:10087800051545EA16754FEA06164FEAC30343EA1B
:1008880052734FEAC2025FEA1C1CC0D111F4801FE8
:100898000BD141EA00014FF000004FF0004CB6E7E1
:1008A80011F4801F04BF01430020B4F1FD0C88BF80
:1008B800BCF5E06F3FF6AFAEB5EB030C04BFB6EB8B
:1008C800020C5FEA500C50F1000041EB045170BD7E
:1008D8000EF0004E4EEA113114EB5C04C2BFD4EBAB
:1008E8000C0541EA045170BD41F480114FF0000E2F
:1008F800013C90E645EA060E8DE60CEA135594EAAB
:100908000C0F08BF95EA0C0F3FF43BAF94EA0C0FAD
:100918000AD150EA01347FF434AF95EA0C0F7FF422
:1009280025AF104619462CE795EA0C0F06D152EA76
:1009380003353FF4FDAE1046194622E750EA41065A
:1009480018BF52EA43067FF4C5AE50EA41047FF46B
:100958000DAF52EA43057FF4EBAE12E74FEA4102CE
:10096800B2F1E04324BFB3F5001CDCF1FE5C0DD905
:1009780001F0004C4FEAC0024CEA5070B2F1004F4F
:1009880040EB830008BF20F00100704711F0804F52
:1009980021D113F13872BCBF01F00040704741F417
:1009A80080114FEA5252C2F11802C2F1200C10FA1B
:1009B8000CF320FA02F018BF40F001004FEAC123FF
:1009C8004FEAD32303FA0CFC40EA0C0023FA02F3A3
:1009D8004FEA4303CCE77FEA625307D150EA013379
:1009E8001EBF4FF0FE4040F44000704701F0004049
:1009F80040F0FE4040F40000704700BF53B94AB9C8
:100A0800002908BF00281CBF4FF0FF314FF0FF300E
:100A180000F074B9ADF1080C6DE904CE00F006F8E9
:100A2800DDF804E0DDE9022304B070472DE9F04762
:100A3800089D04468E46002B4DD18A42944669D9BA
:100A4800B2FA82F252B101FA02F3C2F1200120FA9D
:100A580001F10CFA02FC41EA030E94404FEA1C48EB
:100A6800210CBEFBF8F61FFA8CF708FB16E341EAE7
:100A7800034306FB07F199420AD91CEB030306F16D
:100A8800FF3080F01F81994240F21C81023E63448E
:100A98005B1AA4B2B3FBF8F008FB103344EA034432
:100AA80000FB07F7A7420AD91CEB040400F1FF3347
:100AB80080F00A81A74240F207816444023840EA84
:100AC8000640E41B00261DB1D4400023C5E90043BD
:100AD8003146BDE8F0878B4209D9002D00F0EF8040
:100AE8000026C5E9000130463146BDE8F087B3FA73
:100AF80083F6002E4AD18B4202D3824200F2F9805B
:100B0800841A61EB030301209E46002DE0D0C5E95D
:100B1800004EDDE702B9FFDEB2FA82F2002A40F0A9
:100B28009280A1EB0C014FEA1C471FFA8CFE0126AC
:100B3800200CB1FBF7F307FB131140EA01410EFB50
:100B480003F0884208D91CEB010103F1FF3802D2F7
:100B5800884200F2CB804346091AA4B2B1FBF7F0F1
:100B680007FB101144EA01440EFB00FEA64508D914
:100B78001CEB040400F1FF3102D2A64500F2BB8051
:100B88000846A4EB0E0440EA03409CE7C6F12007A0
:100B9800B34022FA07FC4CEA030C20FA07F401FAE6
:100BA80006F31C43F9404FEA1C4900FA06F3B1FB6F
:100BB800F9F8200C1FFA8CFE09FB181140EA0141D4
:100BC80008FB0EF0884202FA06F20BD91CEB010171
:100BD80008F1FF3A80F08880884240F28580A8F1C9
:100BE80002086144091AA4B2B1FBF9F009FB10111B
:100BF80044EA014100FB0EFE8E4508D91CEB0101B9
:100C080000F1FF346CD28E456AD90238614440EA5B
:100C18000840A0FB0294A1EB0E01A142C846A646DB
:100C280056D353D05DB1B3EB080261EB0E0101FA64
:100C380007F722FA06F3F1401F43C5E900710026C1
:100C48003146BDE8F087C2F12003D8400CFA02FC17
:100C580021FA03F3914001434FEA1C471FFA8CFE27
:100C6800B3FBF7F007FB10360B0C43EA064300FB17
:100C78000EF69E4204FA02F408D91CEB030300F1B5
:100C8800FF382FD29E422DD9023863449B1B89B26C
:100C9800B3FBF7F607FB163341EA034106FB0EF3F5
:100CA8008B4208D91CEB010106F1FF3816D28B42A2
:100CB80014D9023E6144C91A46EA004638E72E466E
:100CC800284605E70646E3E61846F8E64B45A9D266
:100CD800B9EB020864EB0C0E0138A3E74646EAE7D5
:100CE800204694E74046D1E7D0467BE7023B614483
:100CF80032E7304609E76444023842E7704700BFEC
:100D080030B595B03022002108A801F067FE002414
:100D18000394049405940694079401941A4B1A6C4E
:100D280042F080521A641B6C03F080530193019BBC
:100D38000294164B1A6842F480421A601B6803F446
:100D480080430293029B0225089501230B931023ED
:100D58000C930E950F940823109348231193129522
:100D68000323139308A800F011FE0F23039304959F
:100D780005944FF4805306930794294603A801F07D
:100D880023F815B030BD00BF0038024000700040A5
:100D980008B55B4B5B4A9A6001F07CFAFFF7B0FF3D
:100DA80000F0D0F800F04CF900F016F900F02EF938
:100DB80001F0D6FA544C204601F002FC32212046BC
:100DC80001F096FC204601F0B9FD10F4007F29D10E
:100DD8004E4C0A23042221464D4800F070FC42F292
:100DE800107001F083FA94ED007AF2EE0C7AB4EE0A
:100DF800E77AF1EE10FADDD5464B1B68002BD9D106
:100E0800454C01224FF40041204601F097F947F282
:100E1800305001F06BFA00224FF40041204601F0F7
:100E28008DF9C7E7204601F0B9FC80B23B4B18802A
:100E380007EE900AB8EEE78ADFED397A28EE278ABE
:100E4800DFED387A28EE278A374B83ED008A374B57
:100E5800D3ED008AB4EEE88AF1EE10FA27DD344BC0
:100E6800D3ED007A77EEE87A17EE900AFFF70CFBDD
:100E780002460B4600202F49FFF788FC04460D4622
:100E880078EE687A17EE900AFFF7FEFA02460B46EC
:100E980020462946FFF750FB02460B46002026490C
:100EA800FFF792F9FFF75AFD184B186090E7234BAC
:100EB800D3ED007A78EEE77A17EE900AFFF7E4FAB6
:100EC80002460B4600201B49FFF760FC04460D460E
:100ED80078EE687A17EE900AFFF7D6FA02460B46C4
:100EE80020462946FFF728FB02460B4600201249F8
:100EF800FFF76AF9FFF732FD044B186068E700BF97
:100F080000ED00E000000108080100203800002082
:100F1800C400002040000020000C024034000020E3
:100F280033335340000080393C0000200800002083
:100F3800040000200000084000001C4000000020C1
:100F48007047000030B58BB00024059406940794D0
:100F58000894099401941E4B1A6B42F001021A631B
:100F68001A6B02F001020192019A02941A6B42F084
:100F780008021A631A6B02F008020292029A03949A
:100F88001A6B42F004021A631A6B02F0040203920D
:100F9800039A04941A6B42F002021A631B6B03F063
:100FA80002030493049B0B4D22464FF470412846DC
:100FB80001F0C4F84FF47043059301230693079496
:100FC800089405A9284600F0D3FF0BB030BD00BF38
:100FD80000380240000C024008B50A480A4B03607A
:100FE8004FF4E133436000238360C36003610C2244
:100FF80042618361C36100F033FB00B908BDFFF7AC
:101008009FFFFBE7C4000020004C004008B50A48D9
:101018000A4B03604FF4E133436000238360C360ED
:1010280003610C2242618361C36100F019FB00B9BE
:1010380008BDFFF785FFFBE74400002000100140D2
:1010480008B50A480A4B03604FF41643436000236F
:101058008360C36003610C2242618361C36100F055
:10106800FFFA00B908BDFFF76BFFFBE7840000201B
:101078000044004010B58CB00023079308930993EF
:101088000A930B930368494A934207D0484A93420C
:1010980032D0484A93425CD00CB010BD0024019471
:1010A800454B1A6C42F400221A641A6C02F40022AE
:1010B8000192019A02941A6B42F004021A631B6BA4
:1010C80003F004030293029B4FF440630793022347
:1010D80008930123099303230A9308230B9307A971
:1010E800364800F045FF22462146342001F052F8E8
:1010F800342001F087F8CFE7002403942E4B5A6C74
:1011080042F010025A645A6C02F010020392039AD9
:1011180004941A6B42F002021A631B6B03F0020379
:101128000493049BC0230793022308930123099384
:1011380003230A9307230B9307A9214800F018FFFC
:1011480022462146252001F025F8252001F05AF8ED
:10115800A2E700240594184B1A6C42F400321A6472
:101168001A6C02F400320592059A06941A6B42F042
:1011780008021A631B6B03F008030693069B60239F
:101188000793022308930123099303230A93072350
:101198000B9307A90B4800F0EBFE224621462620B8
:1011A80000F0F8FF262001F02DF875E7004C00400C
:1011B800001001400044004000380240000802408E
:1011C80000040240000C02407047FEE7FEE7FEE71D
:1011D800FEE770477047704708B501F075F808BD1D
:1011E80008B5024800F03AFB08BD00BF44000020E3
:1011F80008B5024800F032FB08BD00BF840000209B
:1012080008B5024800F02AFB08BD00BFC400002052
:1012180082B0002100910B4B5A6C42F480425A6410
:101228005A6C02F480420092009A01911A6C42F0C2
:1012380080521A641B6C03F080530193019B02B027
:10124800704700BF003802400268D36823F49073E7
:10125800D3600268536923F001035361202380F8A7
:101268003A30704790F83930DBB2212B01D0022098
:1012780070478368B3F5805F17D0036A5A1C02620F
:101288001A7803685A60C38C9BB2013B9BB2C38433
:101298004BB90268D36823F08003D3600268D3682F
:1012A80043F04003D36000207047036A1B8802683C
:1012B800C3F30803536003691BB9036A023303626B
:1012C800E1E7036A01330362DDE700002DE9F84333
:1012D80004460268136923F44053C1680B43136141
:1012E80083680269134342691343C2691A43016858
:1012F800CB6823F4164323F00C031343CB60026836
:10130800536923F4407381690B435361C369B3F58F
:10131800004F5ED00368B54A934200F0108102F591
:101328008062934200F00B8100F002FE00EB800027
:1013380000EB80006568AD00B0FBF5F5AC4FA7FB8E
:1013480005356D092E0100F0F3FD00EB800000EB80
:1013580080006568AD00B0FBF5F500F0E9FD00EB35
:10136800800000EB800063689B00B0FBF3F3A7FBF1
:1013780003235B094FF0640808FB13531B01323346
:10138800A7FB03235B0903F0F003F51800F0D0FD79
:1013980000EB800000EB80006668B600B0FBF6F654
:1013A80000F0C6FD00EB800000EB800063689B0046
:1013B800B0FBF3F0A7FB0030400908FB1060000108
:1013C8003230A7FB0037C7F3431723682F449F60C9
:1013D80009E10368854A93425AD002F58062934234
:1013E80056D000F0A5FD00EB800000EB800065689A
:1013F8006D00B0FBF5F57E4FA7FB05356D094FEA8B
:10140800051900F095FD00EB800000EB8000666890
:101418007600B0FBF6F600F08BFD00EB800000EBE9
:10142800800065686D00B0FBF5F5A7FB05356D0913
:101438004FF0640808FB1565ED003235A7FB05354C
:101448006D096D0005F4F8754D4400F071FD00EB71
:10145800800000EB800066687600B0FBF6F600F0CE
:1014680067FD00EB800000EB800063685B00B0FB69
:10147800F3F3A7FB03235B0908FB1363DB00323399
:10148800A7FB0337C7F3421723682F449F60AAE0DE
:1014980000F05EFD00EB800000EB800065686D00E9
:1014A800B0FBF5F5524FA7FB05356D094FEA051955
:1014B80000F04EFD00EB800000EB800066687600CF
:1014C800B0FBF6F600F044FD00EB800000EB800076
:1014D80065686D00B0FBF5F5A7FB05356D094FF0A4
:1014E800640808FB1565ED003235A7FB05356D0965
:1014F8006D0005F4F8754D4400F02AFD00EB8000FE
:1015080000EB800066687600B0FBF6F600F020FD80
:1015180000EB800000EB800063685B00B0FBF3F336
:10152800A7FB03235B0908FB1363DB003233A7FB2C
:101538000337C7F3421723682F449F6053E000F036
:1015480007FD00EB800000EB80006568AD00B0FB94
:10155800F5F5274FA7FB05356D092E0100F0F8FCBE
:1015680000EB800000EB80006568AD00B0FBF5F58E
:1015780000F0EEFC00EB800000EB800063689B004D
:10158800B0FBF3F3A7FB03235B094FF0640808FBE8
:1015980013531B013233A7FB03235B0903F0F0034A
:1015A800F51800F0D5FC00EB800000EB80006668C1
:1015B800B600B0FBF6F600F0CBFC00EB800000EBC9
:1015C800800063689B00B0FBF3F0A7FB0030400984
:1015D80008FB106000013230A7FB0037C7F3431740
:1015E80023682F449F60BDE8F88300BF00100140C6
:1015F8001F85EB512DE9F84305460F4616469946D7
:10160800DDF820802C68246837EA04030CBF4FF00B
:10161800010C4FF0000CB4451FD1B8F1FF3FF1D0D9
:10162800B8F1000F05D000F05BFEA0EB09004045C3
:10163800E8D92A68D36823F4D073D3602A68536939
:1016480023F001035361202385F8393085F83A30B7
:10165800002385F83830032000E00020BDE8F88337
:1016680058B310B5044690F839300BB3242384F8E6
:1016780039302268D36823F40053D3602046FFF73B
:1016880025FE2268136923F4904313612268536985
:1016980023F02A0353612268D36843F40053D360CC
:1016A8000020E063202384F8393084F83A3010BDF4
:1016B80080F83830FFF7DEFCD8E7012070472DE9C5
:1016C800F04182B01E4690F83930DBB2202B55D15C
:1016D80004460D469046002954D0002A54D090F86C
:1016E8003830012B52D0012380F838300023C363EF
:1016F800212380F8393000F0F3FD0746A4F8248050
:10170800A4F8268010E000963B460022802120465F
:10171800FFF770FF00283BD12B882268C3F308032A
:1017280053602369CBB90235E38C9BB2BBB1E28C21
:1017380092B2013A92B2E284A368B3F5805FE2D034
:1017480000963B46002280212046FFF753FF08BB46
:1017580015F8012B23685A60E6E70135E4E700969F
:101768003B46002240212046FFF744FFA0B9202332
:1017780084F83930002384F8383000E0022002B0C1
:10178800BDE8F0810120FAE70120F8E70220F6E73A
:101798000320F4E70320F2E70320F0E7704708B5D9
:1017A8000168CA6822F04002CA60202280F8392005
:1017B800FFF7F4FF002008BD704708B590F83A30ED
:1017C800DBB2222B46D18368B3F5805F0FD0036963
:1017D8000BBB03685A68836A591C81621A70C38DEF
:1017E8009BB2013B9BB2C385F3B1002008BD826A5E
:1017F800036943B903685B68C3F308031380836A0A
:1018080002338362EBE703685B68DBB21380836AA9
:1018180001338362E3E703685B68826A511C816273
:1018280003F07F031370DAE70268D36823F020031C
:10183800D3600268D36823F48073D3600268536965
:1018480023F001035361202380F83A30FFF7B4FFF7
:101858000020CBE70220C9E77047000010B5044616
:1018680002681368D168526913F00F0005D113F0AC
:10187800200F02D011F0200F13D128B112F001026D
:1018880013D111F4907F10D113F0800F02D011F012
:10189800800F69D113F0400F02D011F0400F67D1CB
:1018A80010BD2046FFF789FFFAE713F0010F06D0B5
:1018B80011F4807F03D0E06B40F00100E06313F087
:1018C800040F04D01AB1E06B40F00200E06313F09B
:1018D800020F04D01AB1E06B40F00400E06313F08B
:1018E800080F04D01AB1E26B42F00802E263E26B1F
:1018F800002AD5D013F0200F02D011F0200F21D1EB
:1019080023685B6903F04003E26B12F0080F00D113
:1019180023B32046FFF798FC23685A6912F0400F5A
:1019280018D05A6922F040025A61636B73B1124AA7
:101938001A65606B00F008FC0028B1D0606B036D7D
:101948009847ADE72046FFF738FFD9E72046FFF76D
:1019580083FFA5E72046FFF77FFFA1E72046FFF7B3
:101968007BFF0023E3639BE72046FFF77BFC97E7B9
:101978002046FFF714FF93E78519010808B5806B27
:101988000023C385C384FFF767FF08BD002800F064
:10199800BA8170B582B00446036813F0010F3BD0DA
:1019A8009F4B9B6803F00C03042B2CD09C4B9B682B
:1019B80003F00C03082B21D06368B3F5803F4FD0A8
:1019C800B3F5A02F52D0964B1A6822F480321A60D1
:1019D8001A6822F480221A606368002B50D000F045
:1019E8007FFC05468E4B1B6813F4003F14D100F0B2
:1019F80077FC401B6428F5D903208BE1884B5B6892
:101A080013F4800FD8D0864B1B6813F4003F03D023
:101A18006368002B00F07981236813F0020F54D01B
:101A28007F4B9B6813F00C0F3ED07D4B9B6803F0F7
:101A38000C03082B33D0E368002B68D0794B0122C4
:101A48001A6000F04DFC0546754B1B6813F0020F39
:101A580054D100F045FC401B0228F5D9032059E178
:101A68006F4A136843F480331360B5E76C4B1A6808
:101A780042F480221A601A6842F480321A60ABE796
:101A880000F02EFC0546664B1B6813F4003FC3D0DC
:101A980000F026FC401B6428F5D903203AE1604B8E
:101AA8005B6813F4800FC6D15D4B1B6813F0020FFF
:101AB80003D0E368012B40F02A81594A136823F0C8
:101AC800F803216943EAC1031360236813F0080F80
:101AD80042D063696BB3534B0122C3F8802E00F0E8
:101AE800FFFB05464E4B5B6F13F0020F34D100F03D
:101AF800F7FB401B0228F5D903200BE1484A13687D
:101B080023F0F803216943EAC1031360DDE7454B7D
:101B180000221A6000F0E4FB0546414B1B6813F0F5
:101B2800020FD2D000F0DCFB401B0228F5D90320BD
:101B3800F0E03C4B0022C3F8802E00F0D1FB0546B4
:101B4800374B5B6F13F0020F06D000F0C9FB401B48
:101B58000228F5D90320DDE0236813F0040F77D0BD
:101B68002F4B1B6C13F0805F33D1002301932C4B58
:101B78001A6C42F080521A641B6C03F08053019374
:101B8800019B0125284B1B6813F4807F23D0A36891
:101B9800012B34D0052B38D0214B1A6F22F00102CB
:101BA8001A671A6F22F004021A67A368002B3DD047
:101BB80000F096FB06461A4B1B6F13F0020F46D136
:101BC80000F08EFB801B41F288339842F3D9032042
:101BD800A0E00025D6E7144A136843F48073136025
:101BE80000F07EFB0646104B1B6813F4807FCED1B5
:101BF80000F076FB801B0228F5D903208AE0084A0A
:101C0800136F43F001031367CFE7054B1A6F42F0D8
:101C180004021A671A6F42F001021A67C5E700BF8B
:101C280000380240000047420070004000F058FBB6
:101C380006463A4B1B6F13F0020F08D000F050FB1A
:101C4800801B41F288339842F3D9032062E0E5B95A
:101C5800A369002B5DD0314A926802F00C02082A71
:101C68005AD0022B17D02E4B00221A6600F038FBF0
:101C780004462A4B1B6813F0007F42D000F030FB6B
:101C8800001B0228F5D9032044E0244A136C23F0F2
:101C980080531364DCE7224B00221A6600F020FB15
:101CA80005461E4B1B6813F0007F06D000F018FB9A
:101CB800401B0228F5D903202CE0E369226A13436C
:101CC800626A43EA8213A26A5208013A43EA02436B
:101CD800E26A43EA0263114A5360114B01221A6611
:101CE80000F0FEFA04460D4B1B6813F0007F06D186
:101CF80000F0F6FA001B0228F5D903200AE00020BC
:101D080008E0002006E001207047012002E00120E1
:101D180000E0002002B070BD0120FBE7003802405F
:101D28000000474208B5254B9B6803F00C03042BC1
:101D38003FD0082B3FD1214B5A6802F03F025B6825
:101D480013F4800F12D01D4B5968C1F388111C4839
:101D58000023A1FB0001FEF751FE184B5B68C3F39B
:101D6800014301335B00B0FBF3F025E0134B5968E6
:101D7800C1F3881C4FEA4C11B1EB0C006EEB0E0E50
:101D88004FEA8E1343EA90638101091A63EB0E034D
:101D9800DB0043EA5173C90011EB0C0C43F100035B
:101DA800990200234FEA8C2041EA9C51FEF726FE57
:101DB800D3E7034800E0034808BD00BF00380240ED
:101DC80040787D010024F400002800F09A8070B566
:101DD8000D4604464F4B1B6803F00F038B4208D295
:101DE800CBB24C4A1370136803F00F038B4240F0D8
:101DF8008A80236813F0020F17D013F0040F04D061
:101E0800454A936843F4E0539360236813F0080F3E
:101E180004D0414A936843F4604393603E4A936810
:101E280023F0F003A1680B439360236813F0010FBC
:101E380032D06368012B21D09A1E012A25D9364A4F
:101E4800126812F0020F60D033498A6822F0030248
:101E580013438B6000F044FA06462F4B9B6803F04F
:101E68000C036268B3EB820F16D000F039FA801BBE
:101E780041F288339842F0D9032041E0264A12689B
:101E880012F4003FE0D101203AE0234A126812F030
:101E9800007FD9D1012033E01E4B1B6803F00F03EC
:101EA800AB4207D9EAB21B4B1A701B6803F00F0349
:101EB800AB422CD1236813F0040F06D0164A93685E
:101EC80023F4E053E1680B439360236813F0080F91
:101ED80007D0114A936823F46043216943EAC10398
:101EE8009360FFF71FFF0C4B9B68C3F303130B4A68
:101EF800D35CD8400A4B1860002000F0A5F90020F8
:101F080070BD012070470120FAE70120F8E70120A1
:101F1800F6E700BF003C0240003802400C2A0108E6
:101F280014000020014B1868704700BF14000020FF
:101F380008B5FFF7F7FF044B9B68C3F38223034AF6
:101F4800D35CD84008BD00BF003802401C2A0108F5
:101F580008B5FFF7E7FF044B9B68C3F34233034A16
:101F6800D35CD84008BD00BF003802401C2A0108D5
:101F780000230F2B00F2D880F0B583B03AE0072297
:101F880000E00022AA4032430234684D45F824207C
:101F9800674A14686FEA0C0224EA0C054E6816F4C6
:101FA800803F01D04CEA0405614C2560646802EA70
:101FB80004054E6816F4003F01D04CEA04055C4C59
:101FC8006560A46802EA04054E6816F4801F01D013
:101FD8004CEA0405564CA560E46822404D6815F4A7
:101FE800001F01D04CEA0402514CE26001330F2B70
:101FF80000F2988001229A400C6804EA020C32EA46
:102008000404F3D14C68022C01D0122C10D1DD0845
:10201800083550F8257003F00704A6000F24B440D3
:1020280027EA040E0C69B44044EA0E0440F825403F
:1020380006684FEA430E032404FA0EF4E54326EA41
:1020480004064C6804F0030404FA0EF434430460F4
:102058004C68661E012E03D9112C01D0122C0FD109
:1020680086682E40CC6804FA0EF4344384604468D1
:1020780024EA02024C68C4F300149C4014434460F0
:10208800C26815408A6802FA0EF22A43C2604A689A
:1020980012F0805FAAD000220192264A546C44F4C0
:1020A80080445464526C02F480420192019A9C0864
:1020B800A51C1E4A52F8256003F0030295000F2262
:1020C800AA4026EA02061C4A90423FF45AAF02F59B
:1020D800806290421AD002F58062904218D002F5D0
:1020E8008062904216D002F58062904214D002F5C8
:1020F8008062904212D002F58062904210D002F5C0
:10210800806290423FF43BAF08223BE7012239E767
:10211800022237E7032235E7042233E7052231E7B5
:1021280006222FE703B0F0BD704700BF003801401A
:10213800003C014000380240000002400AB18161C1
:10214800704709048161704790F83530DBB2022B83
:1021580003D08023436501207047052380F835307C
:102168000268136823F00103136000207047000021
:10217800074AD36823F4E0631B041B0C000200F435
:10218800E060034343F0BF6343F40033D360704718
:1021980000ED00E000B5194BDB68C3F30223C3F17F
:1021A800070CBCF1040F28BF4FF0040C03F1040E18
:1021B800BEF1060F18D9033B4FF0FF3E0EFA0CFC98
:1021C80021EA0C0199400EFA03F322EA03031943AA
:1021D80000280BDB0901C9B200F1604000F561403D
:1021E80080F800135DF804FB0023E5E700F00F001A
:1021F8000901C9B2024B1954F4E700BF00ED00E031
:1022080014ED00E0002807DB00F01F02400901235D
:102218009340024A42F82030704700BF00E100E0D6
:102228000138B0F1807F0BD24FF0E0235861054AA6
:10223800F02182F823100020986107221A61704764
:102248000120704700ED00E010B504460E4B1878E9
:102258004FF47A73B3FBF0F30C4A1068B0FBF3F059
:10226800FFF7DEFF68B90F2C01D901200AE0002230
:1022780021464FF0FF30FFF78DFF054B1C60002013
:1022880000E0012010BD00BF0C0000201400002059
:102298001000002008B50B4B1A6842F400721A604F
:1022A8001A6842F480621A601A6842F480721A60EE
:1022B8000320FFF75DFF0020FFF7C6FFFEF7A8FF2A
:1022C800002008BD003C0240034A1168034B1B78FC
:1022D8000B441360704700BF040100200C0000206D
:1022E800014B1868704700BF0401002038B5044648
:1022F800FFF7F6FF0546B4F1FF3F02D0044B1B7809
:102308001C44FFF7EDFF401BA042FAD338BD00BFC5
:102318000C0000200F49D1F8883043F47003C1F84D
:1023280088300D4B1A6842F001021A60002098604C
:102338001A6822F0847222F480321A60074A5A60BE
:102348001A6822F480221A60D8604FF000638B600C
:10235800704700BF00ED00E0003802401030002454
:1023680000B585B0002300930193029303931448AA
:10237800144A0260436083600361037680F820306A
:10238800C362114A8262C3600122C26180F83030A0
:10239800426100F0E9F868B904230093012301932E
:1023A800002302936946064800F0FCF928B905B0F5
:1023B8005DF804FBFEF7C4FDEEE7FEF7C1FDF6E7A6
:1023C80008010020002001400100000F00B589B07D
:1023D800002303930493059306930793026803F17C
:1023E800804303F590339A4202D009B05DF804FBAC
:1023F8000021019103F58C335A6C42F480725A64BF
:102408005A6C02F480720192019A02911A6B42F09E
:1024180001021A631B6B03F001030293029B102352
:1024280003930323049303A90148FFF7A1FDDCE705
:10243800000002404A4B5A6822F440325A605A68F7
:1024480041680A435A600268536823F480735360F2
:1024580002685368016943EA0123536002685368BC
:1024680023F0407353600268536881680B435360DC
:102478000268936823F40063936002689368C168F4
:102488000B439360826A374B9A4257D0026893682D
:1024980023F07063936002689368816A0B439360CA
:1024A8000268936823F04053936002689368C16A96
:1024B8000B4393600268936823F0020393600268F9
:1024C8009368017E43EA4103936090F82030002B23
:1024D8003FD00268536843F400635360026853684E
:1024E80023F46043536001684B68426A013A43EA47
:1024F80042334B600268D36A23F47003D3620168E5
:10250800CB6AC269013A43EA0253CB620268936814
:1025180023F4007393600268936890F8301043EADC
:10252800412393600268936823F480639360026890
:102538009368416943EA812393607047026893680E
:1025480023F0706393600268936823F040539360AC
:10255800B0E70268536823F400635360CAE700BF1A
:10256800002301400100000F38B310B50446036C86
:1025780043B1236C13F0100F0BD00120002384F813
:102588003C3010BDFFF722FF0023636484F83C3021
:10259800EFE7236C23F4885323F0020343F002038C
:1025A80023642046FFF746FF00206064236C23F075
:1025B800030343F001032364E0E7012070470000B0
:1025C80082B00023019390F83C30012B7DD0012389
:1025D80080F83C3003689A6812F0010F13D19A68AA
:1025E80042F001029A603D4B1B683D4AA2FB03235F
:1025F8009B0C03EB4303019302E0019B013B019316
:10260800019B002BF9D10268936813F0010F5ED08B
:10261800036C23F4E06323F0010343F48073036441
:10262800536813F4806F05D0036C23F4405343F4CC
:1026380080530364036C13F4805F1BD0436C23F056
:1026480006034364002380F83C306FF022031360D4
:10265800244B5B6813F01F0F27D10368224A93426B
:1026680011D002F58072934207D0204A934214D0C9
:1026780000202DE000234364E4E702F5007252686D
:1026880012F01F0FF1D19A6812F0405F22D19A68B8
:1026980042F080429A6000201AE002F58072526887
:1026A80012F0100FEFD0002012E003680E4A934298
:1026B80001D000200CE09A6812F0405F0CD19A68B3
:1026C80042F080429A60002002E0022000E00020F0
:1026D80002B070470020FBE70020F9E71400002053
:1026E80083DE1B43002301400020014000220140FB
:1026F80070B504460D4603689A6812F4806F03D0DB
:102708009B6813F4807F19D1FFF7EAFD064623681A
:102718001A6812F0020F1AD1B5F1FF3FF7D025B1B0
:10272800FFF7DEFD801BA842F1D9236C43F00403B8
:102738002364002384F83C3003202CE0036C43F02E
:1027480020030364002380F83C30012023E06FF06D
:1027580012021A60236C43F40073236423689A6896
:1027680012F0405F16D1207EB0B9DA6A12F4700F09
:1027780003D09B6813F4806F0DD1236C23F480730E
:102788002364236C13F4805F05D1236C43F00103A9
:10279800236400E0002070BD0020FCE70368D86CCB
:1027A8007047000030B482B00023019390F83C30A9
:1027B800012B00F0BB80012380F83C300B68092B0B
:1027C80041D90468E2689BB203EB43031E3B4FF018
:1027D800070C0CFA03F322EA0303E3600468E268D7
:1027E8000B8803EB43031E3B8D6805FA03F3134381
:1027F800E3604B68062B3DD80468626B03EB8303E8
:10280800053B4FF01F0C0CFA03F322EA0303636342
:102818000468626B4B6803EB8303053BB1F800C0A7
:102828000CFA03F3134363630268414B9A4251D095
:1028380002683F4B9A4256D0002380F83C30184635
:1028480002B030BC7047046822699BB203EB4303B3
:102858004FF0070C0CFA03F322EA03032361046820
:1028680022690B8803EB43038D6805FA03F31343CE
:102878002361BEE70C2B16D805682A6B03EB83038C
:10288800233B1F2404FA03F322EA03032B6305689E
:102898002A6B4B6803EB8303233B0C8804FA03F38E
:1028A80013432B63C0E70568EA6A03EB8303413BE4
:1028B8001F2404FA03F322EA0303EB620568EA6AB9
:1028C8004B6803EB8303413B0C8804FA03F313437F
:1028D800EB62A9E70B68122BAAD1164A536843F496
:1028E80080035360A4E70B68103B012BA4D8114A5E
:1028F800536843F4000353600B68102B9CD10E4BB4
:102908001B6802F1467202F52E3202F28332A2FBF4
:1029180003239B0C03EB83035B00019302E0019B01
:10292800013B0193019B002BF9D185E7022087E742
:10293800002001400023014014000020006C704773
:10294800DFF834D0002103E00C4B5B5843500431CE
:102958000B480C4B42189A42F6D30B4A02E000236C
:1029680042F8043B094B9A42F9D3FFF7D3FC00F035
:1029780011F8FEF70DFA704700000220342A01080A
:10298800000000201800002018000020500100203E
:10299800FEE7000070B50D4D0D4C641BA410002619
:1029A800A64209D10B4D0C4C00F020F8641BA41072
:1029B8000026A64205D170BD55F8043B984701365C
:1029C800EEE755F8043B98470136F2E72C2A010850
:1029D8002C2A01082C2A0108302A0108024403463F
:1029E800934200D1704703F8011BF9E7F8B500BF1F
:1029F800F8BC08BC9E467047F8B500BFF8BC08BCD8
:042A08009E4670472F
:102A0C000000000000000000010203040607080992
:082A1C000000000001020304A8
:082A240010E0FF7F010000003B
:042A2C00AD010108EF
:042A3000890101080F
:102A34009A99793F85EB01400000C03F01000000F6
:082A4400100000000024F40062
:04000005080129497C
:00000001FF
